:1000000088C00000A1C000009FC000009DC000008B
:100010009BC0000099C0000097C0000095C0000080
:1000200093C0000091C0000090C0000082C4000096
:1000300027C5000089C0000087C0000085C00000FF
:1000400083C0000081C000007FC000007DC00000B0
:100050007BC0000079C0000077C0000043C20000F0
:1000600073C0000071C000006FC000006DC00000D0
:100070006BC000002403540068006500200052009B
:10008000650070006C0069006300610074006F001F
:100090007200000032034D0061006B0065007200C9
:1000A00042006F007400200049006E00640075007B
:1000B000730074007200690065007300000004039F
:1000C000090409023E00020100C0320904000001D7
:1000D0000202010005240001100424020605240682
:1000E0000001070582030800FF09040100020A005D
:1000F00000000705040240000107058302400001DB
:100100001201100102000008C12316B00100010213
:10011000DC0111241FBECFEFD2E0DEBFCDBF11E066
:10012000A0E0B1E0E4EBF0E102C005900D92A8324E
:10013000B107D9F712E0A8E2B1E001C01D92A134E5
:10014000B107E1F76DD0B4C75BCF349920C080917F
:100150003802882391F584E089BD89B5826089BD24
:1001600009B400FEFDCF8091D8008F7D8093D80028
:100170008091D80080688093D8008091E0008E7FC5
:100180008093E00081E0809338028AD316C080918A
:100190003802882391F08091E00081608093E00034
:1001A0008091D8008F778093D8008091D8008062AA
:1001B0008093D80019BC109238021895ECE6F0E054
:1001C000808184608083E8E6F0E0808182608083C3
:1001D0003C98449A84B7877F84BF28E10FB6F8948F
:1001E00020936000109260000FBE88E090E0909332
:1001F000CD008093CC0086E08093CA001092C800A6
:100200002093C900539A5A9A8AB180638AB98BB1F4
:1002100080638BB983D384E085BD5F9A579A089534
:10022000CDDF2FB7F89480EB91E09093310280936B
:10023000300290933302809332022FBF2FB7F8948D
:100240008BE291E09093AC018093AB019093AE016F
:100250008093AD012FBF7894349BB9C08091380250
:10026000882309F4B4C08091E00081608093E000AD
:100270008091D8008F778093D8008091D8008062D9
:100280008093D80019BC10923802A1C09FB7F8948F
:10029000809134029FBF803811F180E091E0B8D6A0
:1002A00097FD1DC0E0913002F09131028083E09112
:1002B0003002F0913102CF01019690933102809388
:1002C000300222E08033920711F4128301839FB73A
:1002D000F894809134028F5F809334029FBF8FB770
:1002E000F894D091AF018FBFA89903C0D13608F41C
:1002F00040C0A89A8091AF01882309F15D98C0930E
:1003000028011DC0E091AD01F091AE016191F09323
:10031000AE01E093AD0181E0EB3AF80721F4F092F1
:10032000AE01E092AD019FB7F8948091AF0181508A
:100330008093AF019FBF80E091E00AD6D150DD23CA
:1003400009F780912801882341F08091280181508C
:1003500080932801882309F45D9A809129018823DC
:1003600041F080912901815080932901882309F46B
:100370005C9A9FB7F894809134029FBF882311F153
:10038000E0913202F09133029191F0933302E093C5
:10039000320222E0E033F20721F41093330200939B
:1003A00032022FB7F8948091340281508093340246
:1003B0002FBF8091C80085FFFCCF9093CE005C9842
:1003C000C093290180E091E014D6FBD407C000EB74
:1003D00011E0C3E08BE2E82E81E0F82E8091380234
:1003E0008823E1F353CF80E091E068C580E091E09D
:1003F000FBC40F931F93CF938C01FC0187859089D9
:10040000A189B2898030F1EE9F07F0E0AF07F0E0FC
:10041000BF0711F45F9801C05F9AD8015496EC9120
:100420005497E150E23028F4F0E0EA5EFE4FC081DC
:1004300001C0C0E0F8018389823009F4C860D801A6
:1004400055968C915597873031F0883031F0863051
:1004500029F4C26003C0C46001C0C6601092C90024
:100460001092C8001092CA00F8012785308941898E
:1004700052892030F1EE3F07F0E04F07F0E05F07D0
:1004800081F0DA01C901B695A795979587958058AF
:100490009B47A14EBF4FBC01CD01E8D52150304054
:1004A00002C020E130E03093CD002093CC00C09317
:1004B000CA00F80187859089A189B2898030F1EE60
:1004C0009F07F0E0AF07F0E0BF0711F480E001C044
:1004D00082E08093C80088E98093C900CF911F9182
:1004E0000F9108951F920F920FB60F9211242F9320
:1004F0008F939F93EF93FF938091CE009EB39430A0
:10050000F9F4E091AB01F091AC018083E091AB0193
:10051000F091AC01CF0101969093AC018093AB01B7
:1005200021E08B3A920721F48BE291E09283818360
:100530009FB7F8948091AF018F5F8093AF019FBF09
:10054000FF91EF919F918F912F910F900FBE0F9080
:100550001F9018950895923029F0933041F0913012
:10056000E9F417C08EE390E0E2ECF0E01BC08130CC
:1005700041F0813018F0823089F406C0EEEBF0E0F3
:1005800005C0E4E9F0E002C0E4E7F0E0849190E027
:1005900009C082E190E0E0E0F1E004C080E090E09A
:1005A000E0E0F0E0DA011196FC93EE930895AC01DF
:1005B00028E030E080E003C08F5F220F331F241754
:1005C0003507D0F38295807F08958093E900EBEEA4
:1005D000F0E0808181608083EDEEF0E01082609336
:1005E000EC0040838091EE00881F8827881F0895C3
:1005F0001092F40080E08093E9001092F0001092D5
:10060000E8001092ED009091EB009E7F9093EB003C
:100610008F5F853081F708958091390287FF11C07F
:1006200003C08EB38823B1F08091E80082FFF9CF38
:100630008091E8008B778093E80008958EB388233B
:1006400049F08091E80080FFF9CF8091E8008E7733
:100650008093E800089585E69091EC0090FF05C036
:100660009091E80090FF05C01BC09091E80092FDBA
:1006700017C09EB39923B1F09EB39530A9F0909125
:10068000EB0095FD13C09091E10092FFE5CF9091B2
:10069000E1009B7F9093E1008150F1F684E00895A2
:1006A00080E0089582E0089583E0089581E0089550
:1006B00020913F02309140022617370720F4B901FC
:1006C000FC0190E032C061157105D1F72091E8007E
:1006D0002E772093E800F4CF8091E80083FD37C0A7
:1006E0008091E80082FD2DC08EB38823A1F18EB3E6
:1006F000853079F18091E80080FF17C08091F20089
:1007000006C091919093F100615070408F5F611528
:10071000710511F08830A8F391E0883009F090E07D
:100720008091E8008E778093E80061157105A1F64D
:10073000992391F606C08EB3882369F08EB3853075
:1007400061F08091E80082FFF6CF80E0089581E0BB
:10075000089583E0089582E0089583E0089520914C
:100760003F02309140022617370720F4B9019C015F
:1007700090E035C061157105D1F72091E8002E7722
:100780002093E800F4CF8091E80083FD3AC0809187
:10079000E80082FD30C08EB38823B9F18EB3853076
:1007A00091F18091E80080FF1AC08091F20009C0A9
:1007B000F9012F5F3F4FE491E093F10061507040E9
:1007C0008F5F6115710511F0883090F391E08830EA
:1007D00009F090E08091E8008E778093E800611541
:1007E000710589F6992379F606C08EB3882369F0DE
:1007F0008EB3853061F08091E80082FFF6CF80E013
:10080000089581E0089583E0089582E0089583E0EB
:1008100008956115710529F42091E8002B77209344
:10082000E800382F292F24C08091E80083FD30C0D4
:100830008EB3882389F18EB3853061F18091E80011
:1008400082FFF2CFE32FF22F08C08091F100819355
:100850003E2F2F2F6150704031F03E2F2F2F80916F
:10086000F200882391F78091E8008B778093E8006D
:1008700061157105C9F606C08EB3882369F08EB381
:10088000853061F08091E80080FFF6CF80E0089528
:1008900081E0089583E0089582E0089583E008955B
:1008A00042D044D01EBA10923702109236021092F3
:1008B000350284E089BD89B5826089BD09B400FE36
:1008C000FDCF8091D800982F9F779093D8008068B3
:1008D0008093D800809163008E7F80936300809125
:1008E000D8008F7D8093D8008091E0008E7F809328
:1008F000E0008091E1008E7F8093E1008091E20032
:1009000081608093E2008091E100877F8093E10025
:100910008091E20088608093E2000895C1DF81E069
:100920008093380208951092E20008951092E10039
:1009300008951F920F920FB60F9211242F933F9399
:100940004F935F936F937F938F939F93AF93BF93D7
:10095000EF93FF938091E10080FF1BC08091E20044
:1009600080FF17C08091E1008E7F8093E10080912D
:10097000E2008E7F8093E2008091E20080618093AC
:10098000E2008091D80080628093D80019BC1EBA22
:1009900017D28091E10084FF29C08091E20084FF9A
:1009A00025C084E089BD89B5826089BD09B400FE97
:1009B000FDCF8091D8008F7D8093D8008091E10099
:1009C0008F7E8093E1008091E2008F7E8093E20031
:1009D0008091E20081608093E20080913702882359
:1009E00011F084E001C081E08EBBEAD18091E1008A
:1009F00083FF27C08091E20083FF23C08091E10044
:100A0000877F8093E10082E08EBB10923702809155
:100A1000E1008E7F8093E1008091E2008E7F8093E1
:100A2000E2008091E20080618093E200E1DD80E0FD
:100A300060E042E0CADD8091F00088608093F000C1
:100A4000BFD18091E10082FF0AC08091E20082FF65
:100A500006C08091E1008B7F8093E100B1D1FF91CE
:100A6000EF91BF91AF919F918F917F916F915F9126
:100A70004F913F912F910F900FBE0F901F9018959F
:100A80001F920F920FB60F921124EF92FF920F93C5
:100A90001F932F933F934F935F936F937F938F9306
:100AA0009F93AF93BF93EF93FF93CF93DF930F92F7
:100AB000CDB7DEB789EEE82EF12CF7018081877083
:100AC000108200EF10E0F8019081977F9083789476
:100AD000898322D0F894F7011082F8019081986000
:100AE00090838981F70180830F90DF91CF91FF91EF
:100AF000EF91BF91AF919F918F917F916F915F9196
:100B00004F913F912F911F910F91FF90EF900F9078
:100B10000FBE0F901F9018951F93CF93DF93CDB703
:100B2000DEB7AC970FB6F894DEBF0FBECDBF80E046
:100B3000E9E3F2E09091F10091938F5F8830D1F773
:100B40008091390220913A02253009F484C0263080
:100B500040F42130A1F1213070F0233009F017C1A9
:100B60002EC0283009F4E9C0293009F4F8C0263035
:100B700009F00DC18EC0803821F0823809F007C11C
:100B800008C08091350290913602992371F08260FD
:100B90000CC080913D0287708093E9009091EB003A
:100BA00081E095FF80E01092E9009091E800977F46
:100BB0009093E8008093F1001092F100C9C088235F
:100BC00019F0823009F0E3C090E08F7190700097C7
:100BD00029F08230910509F0DBC00BC080913B0207
:100BE000813009F0D5C0233009F080E080933602CF
:100BF0002CC080913B02882341F520913D02277053
:100C000009F4C6C02093E9008091EB0080FFC0C0CA
:100C100080913A02833021F48091EB00806213C00E
:100C20008091EB0080618093EB0081E090E002C056
:100C3000880F991F2A95E2F78093EA001092EA0044
:100C40008091EB0088608093EB001092E900809126
:100C5000E800877F80C0882309F099C010913B028B
:100C60008091E800877F8093E800D6DC04C08EB3D3
:100C7000882309F48DC08091E80080FFF8CF1F77AA
:100C800011F083E001C082E08EBB10681093E30096
:100C90007FC08058823008F07AC080913B029091EA
:100CA0003C0223E08C3D920789F583E08C838AE245
:100CB0008B833FB7F894DE01159680E090E02EE03C
:100CC00041E2E22FF0E040935700E49180FF03C03F
:100CD000E295EF702F5FEF705E2F505D5A3308F092
:100CE000595F5C9311961C9211971296019684316C
:100CF000910539F73FBF8091E800877F8093E80036
:100D0000CE0103966AE270E0D3DC11C060913D022F
:100D1000AE014F5F5F4F1FDCBC010097C9F18091AE
:100D2000E800877F8093E80089819A8118DD8091AF
:100D3000E8008B778093E8002BC0803841F58091E4
:100D4000E800877F8093E800809137028093F1006C
:100D50008091E8008E778093E8005EDC19C08823DC
:100D6000B1F490913B02923098F48091E800877F33
:100D70008093E800909337024FDC809137028823FC
:100D800011F084E001C083E08EBB2DDB01C02EDBBF
:100D90008091E80083FF0AC08091EB00806280931D
:100DA000EB008091E800877F8093E800AC960FB657
:100DB000F894DEBF0FBECDBFDF91CF911F91089594
:100DC0000895CF938EB3882361F0C091E900C77076
:100DD0001092E9008091E80083FF01C09DDEC0937E
:100DE000E900CF9108950895CF93DF93EC018091AE
:100DF000E80083FF60C0888190E020913D0230913F
:100E00003E022817390709F056C080913A02813214
:100E100061F0823220F4803209F04DC019C0823274
:100E200069F1833209F047C038C080913902813AB4
:100E300009F041C08091E800877F8093E800CE01EF
:100E40000F9667E070E034DC8091E8008B7713C088
:100E500080913902813279F58091E800877F809313
:100E6000E800CE010F9667E070E0D3DCCE01C1DA76
:100E70008091E8008E778093E8001DC08091390250
:100E80008132C9F48091E800877F8093E8008091E7
:100E90003B028D87CE015EDB0DC08091390281322D
:100EA00051F48091E800877F8093E800CE01609143
:100EB0003B0299DFB1DBDF91CF9108950F931F9330
:100EC000CF93DF93EC010D96FC0189E0DF011D92C9
:100ED0008A95E9F72A813B8109818C81882311F069
:100EE00014E001C010E0C90162DB412F482B4260D1
:100EF000802F61E86ADB813029F52E813F810D81E9
:100F00008885882311F014E001C010E0C9014FDB8F
:100F1000412F482B4260802F60E857DB813091F4ED
:100F20002A853B8519858C85882311F0C4E001C092
:100F3000C0E0C9013CDB4C2F482B4260812F61ECA3
:100F400044DB01C080E0DF91CF911F910F910895A4
:100F5000CF93FC01C62F8EB38430E1F447855089CE
:100F600061897289411551056105710599F0818189
:100F70008093E9008091E80085FD08C08091E80039
:100F80008E778093E80067DB882329F4C093F10013
:100F900080E001C082E0CF910895FC018EB38430DF
:100FA00011F547855089618972894115510561059F
:100FB0007105C9F081818093E9008091F200882356
:100FC000A1F09091E8008091E8008E778093E8008E
:100FD00095FD0DC040DB882359F49091E8009E7781
:100FE0009093E800089582E0089580E0089580E0FD
:100FF00008952EB3243059F4FC0147855089618946
:101000007289411551056105710509F0C6CF089532
:10101000FC018EB3843021F547855089618972893E
:101020004115510561057105D9F085818093E9006D
:101030008091E80082FF17C08091F200882321F0A0
:101040008091F10090E002C08FEF9FEF2091F200BD
:10105000222359F42091E8002B772093E80008958B
:101060008FEF9FEF08958FEF9FEF0895A1E21A2E63
:10107000AA1BBB1BFD010DC0AA1FBB1FEE1FFF1F3C
:10108000A217B307E407F50720F0A21BB30BE40B8C
:10109000F50B661F771F881F991F1A9469F76095D3
:1010A0007095809590959B01AC01BD01CF0108958D
:0410B000F894FFCFE2
:1010B400000340000004400000020800000000009B
:1010C4000000000000003020A1200000000001000A
:0810D400A10100000000000072
:00000001FF
